:0200000480007A
:100000006F00C0006F2080306F20403093000000F0
:10001000130100009301000013020000930200008E
:100020001303000093030000130400009304000076
:10003000130500009305000013060000930600005E
:100040001307000093070000130800009308000046
:100050001309000093090000130A0000930A00002E
:10006000130B0000930B0000130C0000930C000016
:10007000130D0000930D0000130E0000930E0000FE
:10008000130F0000930F00009702000093820201FB
:10009000739052307350447497020000938202F7B9
:1000A0007390523017C100001301C1ECF32240F1EC
:1000B0009392C2003301510073100134EF20101CE1
:1000C000173500001305059D6F20007D832245082C
:1000D0007390121483204500032185008321C500FD
:1000E0000322050183224501032385018323C501E2
:1000F00003240502832445028325C5020326050344
:1001000083264503032785038327C50303280504A6
:1001100083284504032985048329C504032A05058A
:10012000832A4505032B8505832BC505032C05066E
:10013000832C4506032D8506832DC506032E050752
:10014000832E4507032F8507832FC50703258502C7
:100150007300201073110114232211002326310093
:1001600023284100232A5100232C6100232E7100F3
:1001700023208102232291022324A1022326B102FB
:100180002328C102232AD102232CE102232EF102CB
:1001900023200105232211052324210523263105CF
:1001A00023284105232A5105232C6105232E71059F
:1001B00023208107232291072324A1072326B107A7
:1001C0002328C107232AD107232CE107232EF10777
:1001D000F312011423245100F322001023205108AC
:1001E000F322101423225108F3223014232451083F
:1001F000F322201423265108130501006F20803FAD
:1010000000000000000000000000000000000000E0
:1010100000000000000000000000000000000000D0
:1010200000000000000000000000000000000000C0
:1010300000000000000000000000000000000000B0
:081040000000000000000000A8
:10200000B367B500B3E7C70093F73700B306C50061
:10201000638407023386C50093070500637ED502FB
:1020200003C705009385150093871700A38FE7FE6C
:10203000E398C5FE67800000E37ED5FE93070500A8
:1020400003A70500938747009385450023AEE7FE6D
:10205000E3E8D7FE6780000067800000130101FFFE
:10206000B367C500232481002326110093F73700AE
:10207000130405003307C500638207026376E50099
:1020800093F5F50FEFF09FFD8320C10013050400C9
:1020900003248100130101016780000093F5F50F0F
:1020A00093968500B386B60093970601B386F60033
:1020B000E37CE5FC930705009387470023AED7FE3A
:1020C000E3ECE7FE8320C100130504000324810034
:1020D000130101016780000083470500638E07003C
:1020E0009307050003C7170093871700E31C07FE3B
:1020F0003385A7406780000013050000678000005B
:1021000083470500938515001305150003C7F5FFE8
:1021100063880700E386E7FE3385E74067800000B9
:10212000930700006FF05FFFB367B50093F73700C8
:10213000639E07021378C6FF330805016378050321
:10214000930705006F0000019387470093854500C2
:1021500063F8070183A6070003A70500E386E6FEF0
:102160003385A7403306A640138507003386C50094
:102170006F00400103C705008347F5FF93851500F5
:10218000639AE70013051500E396C5FE13050000EA
:10219000678000003385E7406780000093070500F3
:1021A00003C705009387170093851500A38FE7FEEB
:1021B000E31807FE6780000003470500930600024E
:1021C000930705006318D70003C71700938717000C
:1021D000E30CD7FE9306D0026300D7069306B00245
:1021E0006300D70483C607009305000063820604DA
:1021F000130500009387170013172500138606FDAB
:1022000083C607003307A700131717003305E6003E
:10221000E39206FE638005023305A040678000005C
:1022200083C617009305000093871700E39206FC0E
:10223000130500006780000083C617009305100097
:1022400093871700E39606FA130500006FF09FFED0
:10225000834505006380050697F6FFFF938686DABF
:1022600017F6FFFF130606DE03A7060083A7460046
:1022700013880500130515003367F700B70801013F
:1022800063020702130700002320E6009307000003
:102290002322F60003A7060083A746003367F70052
:1022A000E31207FE23A0060123A2160183450500C1
:1022B000E39C05FA6780000097F6FFFF938686D4BB
:1022C00003A7060083A74600130805009358F541AD
:1022D0003367F7006306070217F6FFFF130686D67B
:1022E000130700002320E600930700002322F600D6
:1022F00003A7060083A746003367F700E31207FE33
:1023000023A0060123A216016F000000130101FFA4
:102310001305903423261100EFF01FFA130101FE7C
:102320001306C1001307B101130390006F00800072
:10233000138707009377F500B337F300B307F04036
:1023400093F777029376F50093870703B387F60038
:102350002300F7009396C501135545009307F7FF37
:1023600033E5A60093D54500E314E6FC0345C10020
:10237000230E0100630205069305060097F6FFFF92
:10238000938646C817F6FFFF1306C6CB03A70600C1
:1023900083A7460013080500938515003367F700EF
:1023A000B708010163020702130700002320E600BB
:1023B000930700002322F60003A7060083A7460028
:1023C0003367F700E31207FE03C5050023A00601EB
:1023D00023A21601E31C05FA130101026780000025
:1023E000130101FD9307100037F7FFFF2326F100CB
:1023F0002326110223248102232291022320210378
:10240000232E3101232C4101232A510123240100D1
:10241000B306E500B7E7030063F6F6189359C50065
:1024200093840940174900001309C9BD93972400FC
:10243000B307F90083A707003374E500639607101C
:1024400017670000130747BC032A070063000A1838
:1024500083274A009766000083A6C6BA2320F700A8
:10246000638CD7121306C100930581001305040085
:10247000832A0A00EF0040616310051093D6CA005A
:102480009396A60093E6F60193972400B307F9000C
:1024900013E7060C23A0E70073000412973700002F
:1024A000938747B693993900B387370103A707008D
:1024B0006318071203270A00B705040023A0E700EA
:1024C00003274A0023A2E700F3A50510B707C0FFC2
:1024D000B307F40037160000130704003386C70063
:1024E00003A3070083A8470003A8870003A5C7002C
:1024F0002320670023221701232407012326A70096
:102500009387070113070701E39CC7FC739005102D
:1025100093972400B304F90023A0D400730004129D
:102520000F1000008320C102032481028324410292
:10253000032901028329C101032A8101832A410160
:10254000130101036780000013F707046302070407
:1025500013F70708631207061307F00093E707084D
:10256000639CE50493942400B304990023A0F40031
:10257000730004126FF01FFB83260A00832781007B
:1025800093D6C6009396A600B3E6F6006FF0DFEF91
:1025900093E707046FF01FFD9767000023A407A6C9
:1025A0006FF05FEC17150000130505A0EFF05FCA90
:1025B00013053000EFF05FD017150000130505A3D9
:1025C000EFF01FC913053000EFF01FCF1715000003
:1025D000130545A6EFF0DFC713053000EFF0DFCDA0
:1025E00017150000130585A6EFF09FC613053000F0
:1025F000EFF09FCC130101FB232481042326110457
:102600002322910423202105232E3103232C41036F
:10261000232A5103232861032326710323248103E2
:10262000232291032320A103232EB10113040500CB
:10263000EF000045631205108325C408930780004E
:102640006380F512930720006380F506938745FFAA
:10265000130710006376F7009307F000639CF520E2
:1026600003258408EFF0DFD7130504000324810459
:102670008320C10483244104032901048329C10365
:10268000032A8103832A4103032B0103832BC10205
:10269000032C8102832C4102032D0102832DC101F1
:1026A000130101056FD09FA20327440893773700D9
:1026B000639E0708EF0780007310300003270700B0
:1026C00083A707006300F70813051004971500009F
:1026D0009385859B97F6FFFF9386C69217F6FFFFBB
:1026E0001306469603A7060083A7460013090500B4
:1026F000938515003367F700B709010163020702EC
:10270000930700002320F60013080000232206018F
:1027100003A7060083A746003367F700E31207FE0E
:1027200003C5050023A0260123A23601E31C05FAF8
:1027300013053000EFF05FB813050400EFD01F99C8
:102740006FF09FEF13051000EFF01FB71715000093
:102750001305C59CEFF0DFAF13053000EFF0DFB5D8
:102760008327840237190000973A0000938A8A89E8
:102770002326F100174D0000130DCD88B70C04007F
:10278000370CC0FF176A0000130ACA87976B000056
:10279000938B8B8737FB03009357C90093993700BE
:1027A00033873A0103270700630C07089387074024
:1027B00093972700B307FD0083A4070093F7040451
:1027C0006380070AF3AD0C1033048901371600004B
:1027D0009305040013050900EFF01F956304050439
:1027E00093F404086380040AB71600001307090075
:1027F00093070400B306D900032807000325470008
:10280000832587000326C70023A0070123A2A70072
:1028100023A4B70023A6C700130707019387070166
:10282000E31CD7FCB3873A0173900D1003270A000D
:1028300023A00700630007022322F7002320FA00E9
:10284000B71700003309F900E31869F50325C10043
:10285000EFF09FA62320FA0023A0FB006FF05FFE9D
:102860001715000013050585EFF09F9E1305300036
:10287000EFF09FA4171500001305858CEFF05F9D06
:102880006FF01FEB1715000013050586EFF05F9C36
:1028900013053000EFF05FA2F32740F163960716AF
:1028A00017460000130606769357C600130101F67B
:1028B0009397A700232E1108232C81089735000039
:1028C0009385457493E7170023A0F500B707002010
:1028D00093D6C500370700809387F70C232EF6FEAA
:1028E000B3E7E60073900718F3260018639ED71627
:1028F000130405001347F7FF9307F0019702000048
:1029000093824201F39252307310073B7390073A5F
:102910007390523097E7BF7F938707847390571067
:10292000F3270034B708C07FB387170173900714EB
:10293000B7B700009387071073902730B7E70100FF
:102940009387076073900730735040309737C07F8C
:102950009387C78A175700002328F76A9737C07FE5
:102960009387C7A817570000232EF768370308007E
:102970001737000013078788173E0000130E8EA735
:1029800093072002930500001303F3039388880044
:102990001396F50193D61700B366D6003386670009
:1029A000B3C7F600330817011316C60093975700F4
:1029B0002320C7002322070193F70702130787008C
:1029C000B3E7F60093D51500E314EEFC13060009F7
:1029D00093050000130501009737000023AA07A004
:1029E000EFF0CFE7B70700803304F40013050100D0
:1029F00023228108EFD08FED8320C10903248109B0
:102A00001301010A67800000B7F79A0E3706080025
:102A10009387F736130700001306C6FF37080080B8
:102A2000370500406F00C0022FA006009315F70184
:102A300093D61700B3E6D500B3C7D7009397E70145
:102A4000B375F500135717009387060033E7E500C9
:102A5000B3F6C70093F51700B3860601E39605FCAD
:102A600003A006006FF09FFC17050000130505701A
:102A7000EFF00FFE13053000EFF01F8467800000B9
:102A80001305000067800000130500006780000048
:102A900093012000971000009380C0561301A00AF4
:102AA00097070000938747012390200003970000B9
:102AB0006F008000130701009303A00A6316774C90
:102AC00093013000971000009380C05337B1FFFF8F
:102AD000130101A09707000093874701239120006D
:102AE000039720006F00800013070100B7B3FFFFBA
:102AF000938303A0631A7748930140009710000066
:102B0000938040503711EFBE130101AA97070000D0
:102B1000938747012392200003A740006F008000A5
:102B200013070100B713EFBE938303AA631E774414
:102B300093015000971000009380C04C37A1FFFF15
:102B40001301A100970700009387470123932000FA
:102B5000039760006F00800013070100B7A3FFFF19
:102B60009383A300631277429301600097100000E3
:102B70009380204A1301A00A97070000938747011A
:102B8000239D20FE0397A0FF6F0080001307010024
:102B90009303A00A631A773E930170009710000018
:102BA0009380204737B1FFFF130101A09707000072
:102BB00093874701239E20FE0397C0FF6F0080008C
:102BC00013070100B7B3FFFF938303A0631E773A97
:102BD00093018000971000009380A04337110000FC
:102BE000130101AA9707000093874701239F20FE46
:102BF0000397E0FF6F00800013070100B713000088
:102C0000938303AA63127738930190009710000012
:102C10009380204037A1FFFF1301A1009707000018
:102C20009387470123902000039700006F008000E6
:102C300013070100B7A3FFFF9383A3006316773444
:102C40009301A000971000009380C03C37513412CC
:102C500013018167138200FE231022028392000079
:102C6000B753000093838367639072329301B0007F
:102C7000971000009380003A37310000130181095A
:102C80009380B0FFA3932000171200001302A23814
:102C900083120200B7330000938383096396722E78
:102CA0009301C00013020000B7D0FFFF9380D0CD86
:102CB0001711000013010135231011000317010043
:102CC000B7D3FFFF9383D3CD6310772C1302120089
:102CD00093022000E31A52FC9301D000130200007B
:102CE000B7C0FFFF9380D0CC1711000013018131D2
:102CF000130000002311110003172100B7C3FFFFC9
:102D00009383D3CC6312772813021200930220001E
:102D1000E31852FC9301E00013020000B7C0FFFF6C
:102D20009380C0BC171100001301C12D13000000D7
:102D3000130000002312110003174100B7C3FFFF67
:102D40009383C3BC63127724130212009302200002
:102D5000E31652FC9301F00013020000B7B0FFFF2E
:102D60009380C0BB130000001711000013018129DC
:102D70002313110003176100B7B3FFFF9383C3BB95
:102D8000631477201302120093022000E31852FC10
:102D90009301000113020000B7B0FFFF9380B0ABB6
:102DA00013000000171100001301C12513000000DB
:102DB0002314110003178100B7B3FFFF9383B3AB54
:102DC0006314771C1302120093022000E31652FCD6
:102DD0009301100113020000B7E0FFFF9380B0AA37
:102DE00013000000130000001711000013018121DF
:102DF000231511000317A100B7E3FFFF9383B3AAC4
:102E0000631477181302120093022000E31652FC99
:102E10009301200113020000171100001301811E0D
:102E2000B720000093803023231011000317010006
:102E3000B72300009383332363187714130212001F
:102E400093022000E31A52FC9301300113020000A8
:102E5000171100001301011BB710000093803022EE
:102E6000130000002311110003172100B713000005
:102E700093833322631A7710130212009302200007
:102E8000E31852FC930140011302000017110000E7
:102E900013014117B71000009380201213000000A7
:102EA000130000002312110003174100B7130000A4
:102EB00093832312631A770C1302120093022000EB
:102EC000E31652FC93015001130200001711000099
:102ED000130141131300000093002011231311006C
:102EE00003176100930320116310770A1302120085
:102EF00093022000E31C52FC9301600113020000C6
:102F000017110000130101101300000093001001BD
:102F10001300000023141100031781009303100114
:102F2000631477061302120093022000E31A52FC86
:102F30009301700113020000171100001301810CAE
:102F40001300000013000000B73000009380100051
:102F5000231511000317A100B7330000938313005A
:102F6000631477021302120093022000E31652FC4E
:102F700037C500001305F5EE971500009385850809
:102F80002393A500631A3000139511006300050018
:102F90001365150073000000130510007300000096
:042FA000731000C0EA
:102FA400417373657274696F6E206661696C6564E0
:102FB4003A2061646472203E3D202831554C203C07
:102FC4003C203132292026262061646472203C2072
:102FD4003633202A202831554C203C3C20313229DC
:102FE4000A000000417373657274696F6E20666134
:102FF400696C65643A20212870745B315D5B61649F
:1030040064722F2831554C203C3C203132295D20FC
:1030140026203078303830292026262063617573C5
:1030240065203D3D203078660A00000041737365D9
:103034007274696F6E206661696C65643A206E6FA4
:1030440064650A00417373657274696F6E2066610A
:10305400696C65643A20757365725F6D617070693F
:103064006E675B616464722F2831554C203C3C20B0
:103074003132295D2E61646472203D3D20300A00A6
:10308400417373657274696F6E206661696C6564FF
:103094003A202122696C6C6567616C20696E7374D7
:1030A40072756374696F6E220A0000004173736560
:1030B4007274696F6E206661696C65643A2070741D
:1030C4005B315D5B616464722F2831554C203C3C5C
:1030D400203132295D20262030783034300A000037
:1030E400417373657274696F6E206661696C65649F
:1030F4003A2070745B315D5B616464722F283155D2
:103104004C203C3C203132295D2026203078303858
:10311400300A0000417373657274696F6E206661D2
:10312400696C65643A2074662D3E657063202520C1
:1031340034203D3D20300A00417373657274696F19
:103144006E206661696C65643A202122756E65782B
:1031540070656374656420657863657074696F6E07
:10316400220A0000417373657274696F6E20666190
:10317400696C65643A202122756E737570706F7284
:103184007465642073617470206D6F6465220A0035
:10400000EFBEEFBEEFBEEFBEEFBEEFBEEFBEEFBE48
:04401000EFBEEFBE52
:040000058000000077
:00000001FF
